:100000000C942A000C9445000C9445000C94450077
:100010000C9445000C9445000C9445000C9445004C
:100020000C9445000C9445000C9445000C9445003C
:100030000C9445000C9445000C9445000C9445002C
:100040000C9445000C9445000C9445000C9445001C
:100050000C94450011241FBECFE5D4E0DEBFCDBF18
:1000600010E0A0E6B0E0E8EFF4E002C005900D92E9
:10007000A036B107D9F710E0A0E6B0E001C01D92AC
:10008000A036B107E1F70C946B000C940000CF93FD
:10009000DF93CDB7DEB722970FB6F894DEBF0FBE61
:1000A000CDBF1A82198289819A818053954751F078
:1000B00089819A8101969A83898389819A81805363
:1000C0009547B1F722960FB6F894DEBF0FBECDBFAD
:1000D000DF91CF910895CCE5D4E0DEBFCDBF0E9483
:1000E0009B0117B885E886B986B1806586B9349BCF
:1000F000FECF84B195B1880F991F0196AA27BB271F
:10010000BC01CD0128E833E140E050E00E943B0211
:10011000DC01CB012BE0B695A795979587952A959D
:10012000D1F70596A11DB11DBC01CD012AE030E03B
:1001300040E050E00E945A0279018A010E948B013E
:10014000C801B70124E630E040E050E00E945A02C6
:10015000DA01C9012AE030E0AE014F5F5F4FBC0118
:10016000CD010E940602CE0101960E94E5018EE2B9
:100170000E94E201C801B70124E630E040E050E00F
:100180000E945A02DC01CB012AE030E0AE014F5F51
:100190005F4FBC01CD010E9406028E010F5F1F4F11
:1001A000F80101900020E9F73297E017F10719F400
:1001B00080E30E94E201C8010E94E5010E9447001D
:1001C00093CF8150F0F7089581509040E8F708955B
:1001D0001F938AB38E608ABB8AB38F708ABB8BB33E
:1001E000846F8BBBDB9882E00E94E100D99A81E0AA
:1001F0000E94E10019B3107FD99882E00E94E100CB
:10020000D99A81E00E94E10089B382958F70182B02
:10021000D998812F99271F9108951F938AB38E60D3
:100220008ABB8AB38F708ABB8BB38C6F8BBB82E027
:100230000E94E100D99A81E00E94E10019B3107F89
:10024000D99882E00E94E100D99A81E00E94E10001
:1002500089B382958F70182BD998812F99271F9178
:1002600008950E94E8008823E4F3089582E00E9444
:10027000E100D99A81E00E94E100D99808950F9396
:100280001F93082F8AB38E6F8ABB11E08BB3812333
:100290008BBB902F907F8BB3892B8BBB0E94360139
:1002A0008BB381238BBB802F992724E0880F991F64
:1002B0002A95E1F72BB3282B2BBB0E9436010E9415
:1002C00031011F910F9108950F931F93082F8AB347
:1002D0008E6F8ABB11E08BB381238BBB902F907FF5
:1002E0008BB3892B88608BBB0E9436018BB3812333
:1002F0008BBB802F992734E0880F991F3A95E1F73F
:100300002BB3282B28602BBB0E9436010E943101A1
:100310001F910F91089581E00E943F010895882365
:1003200019F08EE090E002C08CE090E0611101963F
:100330000E943F0108951F938AB38E6F8ABB8EEF90
:1003400095E30E94E40011E08BB381238BBB8BB358
:1003500080638BBB0E94360182EC9EE00E94E40029
:100360000E9436018CE590E00E94E4000E94360174
:100370008CE590E00E94E400DC980E9436018CE558
:1003800090E00E94E40088E20E943F0186E00E9423
:100390003F010E948B01612F812F0E948F011F91CD
:1003A000089582E00E943F010895823050F4603148
:1003B00040F48295880F880F807C860F80580E94B9
:1003C0003F0108950E9464010895CF93DF93EC01EB
:1003D0008881882331F089910E94E20188818823F5
:1003E000D1F7DF91CF910895CF93DF93EC01FC011A
:1003F00021968491882339F00E94E201FE01219622
:1004000084918823C9F7DF91CF910895FA01CF93A2
:10041000FF93EF932230CCF02532BCF4C22F2C2F67
:10042000332744275527FF93EF930E945A02EF91F9
:10043000FF91605D6A330CF0695D6193B901CA0197
:10044000605070408040904051F710828F919F9192
:10045000CF910C942B02DC01FC0101900020E9F704
:100460003297AE17BF0730F47C916081708331976B
:100470006D93F7CF0895629FD001739FF001829F23
:10048000E00DF11D649FE00DF11D929FF00D839F23
:10049000F00D749FF00D659FF00D9927729FB00DC0
:1004A000E11DF91F639FB00DE11DF91FBD01CF01D3
:1004B00011240895A1E21A2EAA1BBB1BFD010DC039
:1004C000AA1FBB1FEE1FFF1FA217B307E407F50704
:1004D00020F0A21BB30BE40BF50B661F771F881FE0
:1004E000991F1A9469F760957095809590959B0176
:0804F000AC01BD01CF0108952C
:00000001FF
